BL51 BANKED LINKER/LOCATER V6.00                                                        01/09/2018  11:07:13  PAGE 1


BL51 BANKED LINKER/LOCATER V6.00, INVOKED BY:
C:\KEIL\C51\BIN\BL51.EXE main.obj, Delay_1T.obj TO MA82G5Dxx RAMSIZE (256)


MEMORY MODEL: SMALL WITH FLOATING POINT ARITHMETIC


INPUT MODULES INCLUDED:
  main.obj (MAIN)
  Delay_1T.obj (DELAY_1T)
  C:\KEIL\C51\LIB\C51FPS.LIB (?C?FPMUL)
  C:\KEIL\C51\LIB\C51FPS.LIB (?C?FPDIV)
  C:\KEIL\C51\LIB\C51FPS.LIB (?C?FCAST)
  C:\KEIL\C51\LIB\C51FPS.LIB (?C?FPGETOPN)
  C:\KEIL\C51\LIB\C51S.LIB (?C_STARTUP)
  C:\KEIL\C51\LIB\C51S.LIB (?C?LNEG)


LINK MAP OF MODULE:  MA82G5Dxx (MAIN)


            TYPE    BASE      LENGTH    RELOCATION   SEGMENT NAME
            -----------------------------------------------------

            * * * * * * *   D A T A   M E M O R Y   * * * * * * *
            REG     0000H     0008H     ABSOLUTE     "REG BANK 0"
            DATA    0008H     0010H     UNIT         ?DT?MAIN
                    0018H     0008H                  *** GAP ***
            BIT     0020H.0   0000H.1   UNIT         _BIT_GROUP_
                    0020H.1   0000H.7                *** GAP ***
            IDATA   0021H     0001H     UNIT         ?STACK

            * * * * * * *   C O D E   M E M O R Y   * * * * * * *
            CODE    0000H     0003H     ABSOLUTE     
            CODE    0003H     023CH     UNIT         ?C?LIB_CODE
            CODE    023FH     00A9H     UNIT         CODE_DELAY
            CODE    02E8H     006CH     UNIT         ?PR?MAIN?MAIN
            CODE    0354H     0023H     UNIT         ?PR?_WRITEP?MAIN
            CODE    0377H     0014H     UNIT         ?PR?INITIAL_ADC?MAIN
            CODE    038BH     0012H     UNIT         ?PR?ADC_START?MAIN
            CODE    039DH     000CH     UNIT         ?C_C51STARTUP



OVERLAY MAP OF MODULE:   MA82G5Dxx (MAIN)


SEGMENT                           BIT_GROUP 
  +--> CALLED SEGMENT          START    LENGTH
----------------------------------------------
?C_C51STARTUP                  -----    -----
  +--> ?PR?MAIN?MAIN

?PR?MAIN?MAIN                  -----    -----
  +--> ?PR?INITIAL_ADC?MAIN
  +--> ?PR?ADC_START?MAIN

?PR?INITIAL_ADC?MAIN           -----    -----
BL51 BANKED LINKER/LOCATER V6.00                                                      01/09/2018  11:07:13  PAGE 2


  +--> ?PR?_WRITEP?MAIN

?PR?_WRITEP?MAIN               0020H.0  0000H.1



SYMBOL TABLE OF MODULE:  MA82G5Dxx (MAIN)

  VALUE           TYPE          NAME
  ----------------------------------

  -------         MODULE        MAIN
  C:0000H         SYMBOL        _ICE_DUMMY_
  D:0090H         PUBLIC        P1
  D:00A0H         PUBLIC        P2
  D:00E7H         PUBLIC        ISPCR
  D:00C0H         PUBLIC        XICON
  D:00B0H         PUBLIC        P3
  D:00E8H         PUBLIC        P4
  D:00F8H         PUBLIC        P6
  B:00A8H.7       PUBLIC        EA
  D:00C3H         PUBLIC        ADCFG0
  D:00A8H         PUBLIC        IE
  D:00B8H         PUBLIC        IP0L
  D:00C4H         PUBLIC        ADCON0
  D:00D8H         PUBLIC        CCON
  C:02E8H         PUBLIC        main
  D:00E6H         PUBLIC        SCMD
  D:0008H         PUBLIC        ADC_Value
  D:00E3H         PUBLIC        IFADRH
  D:00E5H         PUBLIC        IFMT
  D:00E4H         PUBLIC        IFADRL
  D:0088H         PUBLIC        TCON
  C:038BH         PUBLIC        ADC_Start
  C:0354H         PUBLIC        _WriteP
  D:000AH         PUBLIC        ADC_Volt
  D:00E2H         PUBLIC        IFD
  D:00C6H         PUBLIC        ADCDH
  D:00C5H         PUBLIC        ADCDL
  D:0098H         PUBLIC        S0CON
  D:000EH         PUBLIC        ADC_Ch0_Value
  D:0010H         PUBLIC        ADC_Ch1_Value
  D:0012H         PUBLIC        VDD_Volt
  D:0016H         PUBLIC        ADC_Ch2_Value
  D:00C8H         PUBLIC        T2CON
  C:0377H         PUBLIC        Initial_ADC
  D:00D0H         PUBLIC        PSW
  -------         PROC          _WRITEP
  D:0007H         SYMBOL        PsfrAddr
  D:0005H         SYMBOL        PsfrData
  -------         DO            
  B:0020H.0       SYMBOL        bEA
  -------         ENDDO         
  C:0354H         LINE#         23
  C:0354H         LINE#         24
  C:0354H         LINE#         25
  C:0358H         LINE#         26
BL51 BANKED LINKER/LOCATER V6.00                                                      01/09/2018  11:07:13  PAGE 3


  C:035AH         LINE#         27
  C:035DH         LINE#         28
  C:035FH         LINE#         29
  C:0361H         LINE#         30
  C:0364H         LINE#         31
  C:0367H         LINE#         32
  C:036AH         LINE#         33
  C:036DH         LINE#         34
  C:036EH         LINE#         35
  C:0370H         LINE#         36
  C:0372H         LINE#         37
  C:0376H         LINE#         38
  -------         ENDPROC       _WRITEP
  -------         PROC          INITIAL_ADC
  C:0377H         LINE#         39
  C:0377H         LINE#         40
  C:0377H         LINE#         41
  C:037AH         LINE#         42
  C:037DH         LINE#         43
  C:0384H         LINE#         44
  -------         ENDPROC       INITIAL_ADC
  -------         PROC          ADC_START
  C:038BH         LINE#         47
  C:038BH         LINE#         48
  C:038BH         LINE#         49
  C:038EH         LINE#         50
  C:0393H         LINE#         51
  C:0396H         LINE#         53
  C:0399H         LINE#         54
  C:039CH         LINE#         55
  -------         ENDPROC       ADC_START
  -------         PROC          MAIN
  C:02E8H         LINE#         57
  C:02E8H         LINE#         58
  C:02E8H         LINE#         60
  C:02EBH         LINE#         63
  C:02EEH         LINE#         64
  C:02F4H         LINE#         66
  C:031BH         LINE#         67
  C:0351H         LINE#         69
  C:0351H         LINE#         70
  C:0351H         LINE#         71
  C:0352H         LINE#         72
  -------         ENDPROC       MAIN
  -------         ENDMOD        MAIN

  -------         MODULE        DELAY_1T
  C:023FH         SEGMENT       CODE_DELAY
  C:02C0H         PUBLIC        DELAY_100US
  C:029FH         PUBLIC        DELAY_10US
  C:0282H         PUBLIC        DELAY_1US
  C:02CBH         PUBLIC        DELAY_200US
  C:02AAH         PUBLIC        DELAY_20US
  C:0285H         PUBLIC        DELAY_2US
  C:02DEH         PUBLIC        DELAY_500US
  C:02B5H         PUBLIC        DELAY_50US
  C:0294H         PUBLIC        DELAY_5US
BL51 BANKED LINKER/LOCATER V6.00                                                      01/09/2018  11:07:13  PAGE 4


  C:023FH         PUBLIC        _DELAY_MS
  D:00E0H         SYMBOL        ACC
  C:026AH         SYMBOL        DELAY_UNIT_1MS
  N:0001H         SYMBOL        FOSC_12MHZ
  N:0000H         SYMBOL        FOSC_24MHZ
  C:024DH         SYMBOL        LSB_LOOP
  C:025AH         SYMBOL        MSB_LOOP0
  C:0257H         SYMBOL        MSB_LOOP1
  C:0253H         SYMBOL        NDLSB
  C:0263H         SYMBOL        NDMSB
  C:023FH         LINE#         29
  C:0241H         LINE#         30
  C:0243H         LINE#         31
  C:0245H         LINE#         33
  C:0247H         LINE#         34
  C:0249H         LINE#         36
  C:024BH         LINE#         37
  C:024DH         LINE#         39
  C:0250H         LINE#         40
  C:0253H         LINE#         42
  C:0255H         LINE#         43
  C:0257H         LINE#         45
  C:025AH         LINE#         47
  C:025DH         LINE#         48
  C:0260H         LINE#         49
  C:0263H         LINE#         51
  C:0265H         LINE#         52
  C:0267H         LINE#         53
  C:0269H         LINE#         54
  C:026AH         LINE#         57
  C:026DH         LINE#         58
  C:0270H         LINE#         59
  C:0273H         LINE#         60
  C:0276H         LINE#         61
  C:0279H         LINE#         62
  C:027CH         LINE#         63
  C:027FH         LINE#         64
  C:0280H         LINE#         65
  C:0281H         LINE#         66
  C:0282H         LINE#         78
  C:0283H         LINE#         78
  C:0284H         LINE#         79
  C:0285H         LINE#         91
  C:0286H         LINE#         91
  C:0287H         LINE#         91
  C:0288H         LINE#         91
  C:0289H         LINE#         91
  C:028AH         LINE#         91
  C:028BH         LINE#         91
  C:028CH         LINE#         91
  C:028DH         LINE#         91
  C:028EH         LINE#         91
  C:028FH         LINE#         91
  C:0290H         LINE#         91
  C:0291H         LINE#         91
  C:0292H         LINE#         91
  C:0293H         LINE#         92
BL51 BANKED LINKER/LOCATER V6.00                                                      01/09/2018  11:07:13  PAGE 5


  C:0294H         LINE#         108
  C:0296H         LINE#         109
  C:0299H         LINE#         110
  C:029CH         LINE#         111
  C:029EH         LINE#         112
  C:029FH         LINE#         127
  C:02A1H         LINE#         128
  C:02A4H         LINE#         129
  C:02A7H         LINE#         130
  C:02A9H         LINE#         131
  C:02AAH         LINE#         146
  C:02ACH         LINE#         147
  C:02AFH         LINE#         148
  C:02B2H         LINE#         149
  C:02B4H         LINE#         150
  C:02B5H         LINE#         165
  C:02B7H         LINE#         166
  C:02BAH         LINE#         167
  C:02BDH         LINE#         168
  C:02BFH         LINE#         169
  C:02C0H         LINE#         184
  C:02C2H         LINE#         185
  C:02C5H         LINE#         186
  C:02C8H         LINE#         187
  C:02CAH         LINE#         188
  C:02CBH         LINE#         206
  C:02CDH         LINE#         207
  C:02D0H         LINE#         208
  C:02D3H         LINE#         209
  C:02D6H         LINE#         210
  C:02D9H         LINE#         211
  C:02DBH         LINE#         212
  C:02DCH         LINE#         212
  C:02DDH         LINE#         213
  C:02DEH         LINE#         234
  C:02E1H         LINE#         235
  C:02E4H         LINE#         236
  C:02E7H         LINE#         237
  -------         ENDMOD        DELAY_1T

  -------         MODULE        ?C?FPMUL
  C:0003H         PUBLIC        ?C?FPMUL
  -------         ENDMOD        ?C?FPMUL

  -------         MODULE        ?C?FPDIV
  C:010CH         PUBLIC        ?C?FPDIV
  -------         ENDMOD        ?C?FPDIV

  -------         MODULE        ?C?FCAST
  C:01B3H         PUBLIC        ?C?FCASTC
  C:01AEH         PUBLIC        ?C?FCASTI
  C:01A9H         PUBLIC        ?C?FCASTL
  -------         ENDMOD        ?C?FCAST

  -------         MODULE        ?C?LNEG
  C:0231H         PUBLIC        ?C?LNEG
  -------         ENDMOD        ?C?LNEG
BL51 BANKED LINKER/LOCATER V6.00                                                      01/09/2018  11:07:13  PAGE 6



Program Size: data=25.1 xdata=0 code=937
LINK/LOCATE RUN COMPLETE.  0 WARNING(S),  0 ERROR(S)
